:100000000C9489000C94360E0C94A8000C94A80053
:100010000C94A8000C94A8000C94A8000C94B70BA6
:100020000C94A8000C94A8000C94A8000C94A800B0
:100030000C94A8000C94A8000C94A8000C94A800A0
:100040000C94A8000C94A8000C94A8000C94A80090
:100050000C94A8000C94A8000C94A8000C94A80080
:100060000C94A8000C94A8000C94A8000C94A80070
:100070000C94A8000C94A8000C94A8000C94A80060
:100080000C94A8000C94A8000C94A8007E09A40964
:10009000B809B809DF09ED09240A9D09B40A7909EC
:1000A0002D0A2F0A390A470A4B0A610A040A6A0A0A
:1000B000860A8D0AB40A940AA00AAD0A090212003F
:1000C000010100C03209040000000000000012011C
:1000D0001001FF000008501DE9600001010200014D
:1000E00012034B00650079006D0061006E00360060
:1000F00034001003480065006E006E0069006E0059
:1001000067002000420065006B0065006C0004037E
:10011000090411241FBECFEFD0E4DEBFCDBF18E02D
:10012000A0E0B1E0E4EBFBE200E00BBF02C007900F
:100130000D92A231B107D9F729E0A2E1B8E001C0E0
:100140001D92A13AB207E1F70E944A0F0C94D8150C
:100150000C940000F999FECF809115089091160833
:1001600092BD81BDF89A809115089091160801966C
:10017000909316088093150880B590E00895F9993A
:10018000FECF209113083091140832BD21BD80BDEF
:10019000FA9AF99A80911308909114080196909315
:1001A00014088093130880E090E0089520915B0884
:1001B00030915C088091590890915A08AC014F5FCA
:1001C0005F4F50935A0840935908F901E80FF91FFF
:1001D000808190E0089592B18091200180958923DB
:1001E00082B992B180912001892B82B9089592B190
:1001F00080912001892B82B992B180912001809554
:10020000892382B90895CF93DF93DC01E0E0F0E029
:1002100090E8EA01888189232D913C9111972E0F56
:100220003F1FEB01882329F08881892339F480E37B
:1002300006C08881892311F488E701C081E3E901C0
:10024000888396953196E830F10519F7ED91FC9188
:10025000119710868D919C91DF91CF910895CF9247
:10026000DF92EF92FF920F931F93CF93DF938C0156
:100270007B016A01C0E0D0E0D80112968D919C917B
:100280001397C817D907C0F4D8011896ED91FC91BF
:100290001997CE01880F991FE80FF91FB7018081C8
:1002A00091810E943B12892B29F4F601D183C083EE
:1002B00081E003C02196E0CF80E0DF91CF911F91D4
:1002C0000F91FF90EF90DF90CF900895CF92DF9243
:1002D000EF92FF920F931F93CF93DF93EC018B016B
:1002E0006A817B81888599856F5F7F4F660F771F55
:1002F0000E943E1199878887C884D984EA80FB8050
:10030000F80101900020E9F7CF0161E070E0801B67
:10031000910B0E940110F701EE0FFF1FEC0DFD1D68
:1003200091838083F80101900020E9F73197AF01B4
:10033000401B510B88859985EA81FB81EE0FFF1FD9
:10034000E80FF91FB801808191810E9444128A81CF
:100350009B8101969B838A838A819B810197DF9190
:10036000CF911F910F91FF90EF90DF90CF90089564
:100370008F929F92AF92BF92EF92FF92CF93DF93B3
:10038000E0E0F0E0E12CF12CEC01AC81BD81EA165B
:10039000FB06C0F4EC01AA85BB85AE0FBF1F8D9094
:1003A0009D90AD90BC90349684169506A606B7062F
:1003B00029F4F901F182E08281E005C0AFEFEA1A89
:1003C000FA0AE2CF80E0DF91CF91FF90EF90BF90EB
:1003D000AF909F908F900895CF92DF92EF92FF920F
:1003E000CF93DF93EC016A017B016C817D818A856B
:1003F0009B856F5F7F4F660F771F660F771F0E9489
:100400003E119B878A878A859B85EC81FD81EE0F53
:10041000FF1FEE0FFF1FE80FF91FC082D182E2829B
:10042000F3828C819D8101969D838C838C819D813B
:100430000197DF91CF91FF90EF90DF90CF900895DB
:100440000F931F93CF93DF93EC018B016881798128
:100450008E819F816F5F7F4F660F771F0E943E11D5
:100460009F838E838E819F81E881F981EE0FFF1F2C
:10047000E80FF91F11830083888199810196998380
:100480008883C801DF91CF911F910F910895FC01DE
:1004900020E030E08081918128173907C8F4A681D7
:1004A000B781A901440F551FA40FB51F0D90BC9132
:1004B000A02D11968C91861308C086819781FC012E
:1004C000E40FF51F8081918108952F5F3F4FE2CFA8
:1004D00080E090E008950E94470221E0892B09F016
:1004E00020E0822F089520E030E0FC01408151811E
:1004F0002417350790F4DC011696ED91FC911797BF
:10050000A901440F551FE40FF51F0190F081E02D64
:10051000438144832F5F3F4FE8CF0895CF93DF930C
:1005200067E070E081E090E00E940110EC0162E081
:1005300070E081E090E00E9401109E838D838091A5
:100540002F06898380E48A8381E08B838C83CE01AC
:10055000DF91CF910895FF920F931F93CF93DF9375
:100560008C01F62E0E946B02811109C06F2DC8010B
:10057000DF91CF911F910F91FF900C9447020E9441
:100580008E02EC01F982BC01C8010E942002CE015A
:10059000DF91CF911F910F91FF900895FC0161832E
:1005A00008950F931F93CF93DF93EC018B01688124
:1005B00070E06F5F7F4F660F771F8D819E810E9475
:1005C0003E118D839E832881FC01E20FF11DE20F15
:1005D000F11D118300832F5F2883C801DF91CF9124
:1005E0001F910F910895FC012381248308950F9397
:1005F0001F93CF93DF938C01C0E0D0E0F8012081FE
:1006000030E085819681C217D30764F49E01220FE2
:10061000331FFC01E20FF31F808191810E94B5100E
:100620002196ECCF0E94B510C801DF91CF911F91A8
:100630000F910C94B5100F931F93CF93DF93EC01A0
:1006400000E010E0288139818E819F810217130715
:1006500068F49801220F331FFC01E20FF31F808121
:1006600091810E94F7020F5F1F4FECCF0E94B510DF
:1006700000E010E02A813B818885998502171307E5
:1006800068F49801220F331FFC01E20FF31F8081F1
:1006900091810E94B5100F5F1F4FECCF0E94B510E3
:1006A0008A859B850E94B510CE01DF91CF911F9165
:1006B0000F910C94B51065E070E081E090E00E942D
:1006C0000110FC0188E0808311828FEF8283838395
:1006D0001482CF0108959F92AF92BF92CF92DF9282
:1006E000EF92FF920F931F93CF93DF93EC0160E49F
:1006F00076E00E94660169E377E0CE010E94660120
:100700006FE277E0CE010E9466010E948E028C01AA
:1007100082E3F80181830E945B03FC018CE0F82EE8
:10072000F08212821382BF01C8010E94D102B80177
:10073000CE010E9420020E945B036C018DE0F60155
:1007400080830E948E028C0183E2F8018183B601CE
:10075000C8010E94D102B801CE010E9420020E946D
:100760008E028C018AE2F80181830E945B03FC0106
:10077000F08281E082831382BF01C8010E94D1020E
:100780009AE0E92EF12C2FE0922E35E2A32E45E0DF
:10079000B42E58EEC52E63E0D62E0E945B03FC01FA
:1007A0009082A382BC01C8010E94D1020E945B0317
:1007B000FC01B082C282D382BC01C8010E94D10276
:1007C000F1E0EF1AF10849F70E945B03FC018CE0AD
:1007D000808382E082831382BF01C8010E94D1021C
:1007E000B801CE010E9420020E948E028C018BE390
:1007F000F80181830E945B03FC0186E18083128201
:100800001382BF01C8010E94D102B801CE010E942B
:10081000200281E0DF91CF911F910F91FF90EF9027
:10082000DF90CF90BF90AF909F9008950F931F934C
:10083000CF93DF93EC018B01CB010E945312982FD1
:10084000991F9927991F9983982F90769C838F7170
:100850008883C8010E9453128A83C8010E945312E0
:100860008B83DF91CF911F910F910895CF92DF92EB
:10087000EF92FF920F931F93CF93DF936C017B0155
:10088000CB010E945312F6018383C7010E945312C9
:1008900000E010E0EC01DD270C171D0764F40E9456
:1008A0005B03BC01C6010E94D102B7010E9416047D
:1008B0000F5F1F4FF1CFDF91CF911F910F91FF90ED
:1008C000EF90DF90CF9008950C94B51064E070E045
:1008D00081E090E00C940110CF93DF936EE070E024
:1008E00081E090E00E940110EC0162E070E081E0A4
:1008F00090E00E9401109F838E83198618861B86C4
:100900001A860E9466049D878C87198218821B8232
:100910001A821D821C82CE01DF91CF9108950F9320
:100920001F93CF93DF93EC018B01CB010E945312F5
:100930008883C8010E9453128983C8010E94531200
:100940008A83C8010E9453128B83DF91CF911F913C
:100950000F9108958F929F92AF92BF92CF92DF92A4
:10096000EF92FF920F931F93CF93DF93CDB7DEB734
:10097000D0510FB6F894DEBF0FBECDBF5C018B0126
:10098000FC01848595850E948F04CE0101964C015F
:10099000C8010E945312F82E80913006F81609F40F
:1009A00063C080912E068F1116C064017601E8188D
:1009B000F908C8010E945312882321F0F60181939F
:1009C0006F01F4CFF401EE0DFF1D1082B401C501DB
:1009D0000E946601DDCF80912D06F81239C0C80152
:1009E0000E9453127C01C8010E9453126C01C8017D
:1009F0000E945312A601DD0C660B770B762F652F34
:100A0000542F4427092E000CAA0BBB0BDC0199279D
:100A10008827842B952BA62BB72B6701FF0CEE089C
:100A2000FF08C82AD92AEA2AFB2AC8010E945312C1
:100A3000AC01990F660B770B742F66275527442757
:100A40004C295D296E297F29C5010E94EC01A0CFA8
:100A50000E948E02BC01C5010E942002FC01F182AD
:100A6000B8010E94360494CF81E0D05F0FB6F894AD
:100A7000DEBF0FBECDBFDF91CF911F910F91FF90D1
:100A8000EF90DF90CF90BF90AF909F908F900895A0
:100A90000F931F93CF93DF9300D0CDB7DEB78C01B8
:100AA000CB0169837A830E94531290913106698148
:100AB0007A8198130BC0CB0169837A830E94531209
:100AC0009091320669817A81981759F090E00E94DE
:100AD0000C1380E00F900F90DF91CF911F910F9139
:100AE0000895C8010F900F90DF91CF911F910F9142
:100AF0000C94AA040C94B510F8949CE088E10FB60D
:100B0000F894A895809360000FBE90936000FFCF8B
:100B100060EB70EB8EEF9FE00E94D3150E947C0586
:100B2000EAE6F8E081E08083118208950E94900552
:100B3000EAE6F8E0128213821482158208950E9478
:100B4000960580911D0180937300E8E6F0E08081B6
:100B500088608083789408950FB6F894A895809162
:100B60006000886180936000109260000FBE8FEF7C
:100B700081B980EC82B989E88AB980EF8BB90C948D
:100B80009F0580E090E0FC01EE0FFF1FEE0FFF1FBE
:100B9000E055F74F1182108201968031910599F747
:100BA0000895CF93DF93882339F026E230E0A8E25E
:100BB000B0E0C7E2D0E006C023E230E0A5E2B0E05A
:100BC000C4E2D0E098E0899FF0011124E62BEE0FFB
:100BD000FF1FEE0FFF1FE055F74F31832083628325
:100BE00043838881962F9095892388838C91682BE5
:100BF0006C93DF91CF910895F8940E94160E519A4C
:100C00002FEF89E698E1215080409040E1F700C045
:100C100000005198789410925C0810925B08089537
:100C200080E090E0FC01EF5CF64F80830196803419
:100C30009105C1F7089585B7806885BF85B780683D
:100C400085BF08959BB180912101892B8BB99BB100
:100C500080912101809589238BB908959BB1809162
:100C60002301892B8BB98AE18A95F1F700C09BB1EA
:100C700080912301809589238BB90895CF92DF92CB
:100C8000FF920F931F93CF93DF931F92CDB7DEB7E1
:100C90000E942206C12CD12C80E0FF24F39486010F
:100CA000085F1F4F29B1909122019223F601E05174
:100CB000F74F911103C0F08281E001C01082898357
:100CC0000E942E069FEFC91AD90A89810C151D05AD
:100CD00049F768010034110511F70F90DF91CF91AA
:100CE0001F910F91FF90DF90CF900895E82FF0E0D3
:100CF000E059F74F9081911111C090911F01662327
:100D000011F0892B02C09095892390912001892BA5
:100D100082B9E0916208F091630809940895CF9335
:100D20009BB180911E01809589238BB98FE99FE04B
:100D30000197F1F700C000009BB180911E01892B43
:100D40008BB9C0E060E08C2F0E947606CF5FC03484
:100D5000C9F7CF910895CF939BB180911E01892B44
:100D60008BB98FE99FE00197F1F700C000009BB1BC
:100D700080911E01809589238BB9C0E060E08C2FA3
:100D80000E947606CF5FC034C9F7CF910895EF92E5
:100D9000FF920F931F93CF93DF931F92CDB7DEB7D0
:100DA000182F062F90E09C012059374F7901F90147
:100DB0008081882319F0808184131DC0F701808110
:100DC000811106C0602F812F49830E9476064981D8
:100DD000011101C040E0F7014083808181110BC007
:100DE000602F812F0F90DF91CF911F910F91FF9076
:100DF000EF900C9476060F90DF91CF911F910F9199
:100E0000FF90EF900895CF93DF93C0E0D0E0FE0114
:100E1000EE0FFF1FEE0FFF1FE055F74F808191810E
:100E2000892BB1F0A081B1819C918281892321F429
:100E3000838142E061E00AC0A381B0E0A059B74FCE
:100E40008C91823029F4838142E060E00E94C706E1
:100E50002196C031D105D9F6DF91CF910895CF9376
:100E6000DF93C0E0D0E0FE01E051F74F6081FE016A
:100E7000EF5CF64F80810E9476062196C034D10542
:100E800091F7DF91CF910895CF93DF931F92CDB764
:100E9000DEB78983898161E00E9476062FEF89EFB2
:100EA00090E0215080409040E1F700C0000089812F
:100EB00060E00F90DF91CF910C947606CF93DF9393
:100EC0001F92CDB7DEB78983E981F0E0E051F74F9B
:100ED00080810F90DF91CF910895CF93DF931F9280
:100EE000CDB7DEB78983E981F0E0E051F74F90811B
:100EF00081E089270F90DF91CF910895CF93DF9301
:100F00001F92CDB7DEB78983998181E0903408F0D4
:100F100080E00F90DF91CF910895CF93DF931F92E0
:100F2000CDB7DEB789838981803410F080E021C09D
:100F30000E943E068823D1F3E981F0E0E051F74FAB
:100F40008081882399F32FEF89EF90E02150804032
:100F50009040E1F700C000000E943E06882331F077
:100F6000E981F0E0E051F74F808102C080E090E03D
:100F700081700F90DF91CF910895CF93DF931F92EF
:100F8000CDB7DEB789838981803410F080E01BC043
:100F90000E943E06E981F0E0E051F74F8081811127
:100FA000F5CF2FEF89EF90E0215080409040E1F79E
:100FB00000C000000E943E06E981F0E0E051F74FDA
:100FC000908181E089270F90DF91CF9108958F92D2
:100FD0009F92AF92BF92CF92DF92FF920F931F9397
:100FE000CF93DF93EC018C01FE0101900020E9F723
:100FF0003197EC1BFD0BC8018C1B9D0B8E179F07B7
:1010000008F04AC0D801ED918D01F0E0CF01880FC2
:10101000991FE80FF91FEC5DFE4FC2808080918020
:101020005401D12CC501881999098C159D05E4F648
:10103000F50181915F01982F907C903849F461E02F
:101040008F730E9476068FE99FE00197F1F70AC03F
:10105000903459F460E08F730E947606AFE9BFE0E8
:101060001197F1F700C00000DDCF903CD9F68F73E7
:10107000F82E80916808F81209C0BFEFE9EFF0E0A0
:10108000B150E040F040E1F700C000008F2D0E9419
:101090004407F0926808C6CFDF91CF911F910F915E
:1010A000FF90DF90CF90BF90AF909F908F9008956A
:1010B000CF93DF93CDB7DEB7D2500FB6F894DEBF33
:1010C0000FBECDBF9E012B5F3D4FF9014191519164
:1010D0009F0160E072E0CE0101960E94D312CE0122
:1010E00001960E94E707DE5F0FB6F894DEBF0FBEE1
:1010F000CDBFDF91CF910895CF92DF92FF920F93F2
:101100001F93CF93DF931F92CDB7DEB780E090E0BF
:10111000FC01E95EF74F1082019680349105C1F71A
:101120000DED17E020E090E0223048F0F801319713
:101130008081803221F4F8018081803289F0FF249F
:10114000F394F90EC92ED12CF801808190E0298307
:101150000E942312F601E95EF74F80839F2D2981BB
:101160002F5F0F5F1F4F2132F9F60F90DF91CF9164
:101170001F910F91FF90DF90CF900895CF93DF9351
:1011800000D0CDB7DEB78FEF97E09A83898388E0F0
:1011900098E00E94E70744E250E065E270E0CE018B
:1011A00001960E9403010E94E7078FE098E00E94E9
:1011B000E7078BE098E00E94E70747E250E068E22B
:1011C00070E0CE0101960E9403010E94E7078EE0C5
:1011D00098E00E94E7070F900F90DF91CF9108955C
:1011E000E0917109F0917209A485B58584B18C9361
:1011F000A485B58585B111968C93A485B58587B1F5
:1012000012968C93A485B58588B113968C9304842B
:10121000F585E02D608182E090E00E94C515E091A7
:101220007109F09172090484F585E02D618183E0F4
:1012300090E00E94C515E0917109F0917209048453
:10124000F585E02D628184E090E00E94C515E09173
:101250007109F09172090484F585E02D638185E0C0
:1012600090E00C94C515E0917109F0917209048425
:10127000F585E02D808184B9E0917109F0917209C2
:101280000484F585E02D818185B9E0917109F091A3
:1012900072090484F585E02D828187B9E091710996
:1012A000F09172090484F585E02D838188B9089551
:1012B000FF920F931F93CF93DF938C01DB01119665
:1012C0008C911197882329F0C8E2D0E027E230E022
:1012D00004C0C5E2D0E024E230E0FC904F2D50E0A5
:1012E0004831510508F040C1FA01EA5BFF4F0C9408
:1012F000F80F13968C918093300936C112964C9159
:101300001297942F50E090FD03C096955F5FFBCF3E
:1013100013968C911397892301C0880F5A95EAF789
:1013200098814095492348839881892B8883F901C6
:10133000908112968C91892BC2C0F90190811296EE
:101340008C911297892B42C0988112968C9112979A
:101350009823F9014081482B4083388112962C91C3
:1013600020952323288328818927822B8883FCC00A
:1013700012965C9112979881452F4923F2E0FF1253
:1013800002C091E001C09FEF852F60E080FD04C0A6
:10139000869546956F5FFACF940F892301C0880F19
:1013A0006A95EAF7F9019081952B9083288112962E
:1013B0009C919095922398839881892BD7CFF9019E
:1013C000908112968C9112978095892380839881C1
:1013D00012968C9180958923C9CF12968D919C91FC
:1013E0001397092E000CAA0BBB0B0097A105B105A2
:1013F00009F4BAC0EFE9FFE03197F1F700C000004F
:101400000197A109B109F1CFF80182859385129660
:10141000ED91FC911397EE0FFF1FEE0FFF1FE80FEA
:10142000F91F80819181A281B3810097A105B10547
:1014300009F49AC0EFE9FFE03197F1F700C000002E
:101440000197A109B109F1CF13968C91DF91CF914A
:101450001F910F91FF900C94570B61E001C060E069
:1014600013968C91DF91CF911F910F91FF900C9467
:101470007606F801808591851296ED91FC9113977F
:10148000EE0FFF1FE80FF91F808191815FC081E09F
:101490008093690869C01296EC911297F0E0EF5CB6
:1014A000F64F80811396CC911397D0E0CF5CD64F46
:1014B000988190831396EC91F0E0EF5CF64F808377
:1014C00053C013968C91DF91CF911F910F91FF9094
:1014D0000C94440713968C91811109C08FE896E013
:1014E00090936508809364088BEE90E00AC0813089
:1014F000D9F58BEA96E0909365088093640887EFAE
:1015000090E090936308809362082EC0DF91CF91A2
:101510001F910F91FF900C94F008DF91CF911F91D4
:101520000F91FF900C94330913964C9113971296D8
:101530006C91DF91CF911F910F91FF900C94D10589
:1015400087E198E00E94E7078EE098E0DF91CF9175
:101550001F910F91FF900C94E707DF91CF911F919E
:101560000F91FF900C94BE08DF91CF911F910F91C6
:10157000FF900895AF92BF92CF92DF92EF92FF92C9
:101580000F931F93CF93DF93EC015B0100E010E01A
:10159000888199810817190708F045C0EE81FF81FD
:1015A0006801CC0CDD1CEC0DFD1D0190F081E02DDF
:1015B000918180912F06981329C0E12CF12C1AC03B
:1015C000EE81FF81EC0DFD1D0190F081E02D058085
:1015D000F681E02DC701880F991FE80FF91F608180
:1015E0007181CE010E945809A114B10491F48FEFCA
:1015F000E81AF80AEE81FF81EC0DFD1D0190F081E3
:10160000E02D808190E0E816F906D4F20F5F1F4FBD
:10161000BFCFC501EFE9FFE03197F1F700C000004F
:101620000197C1F7E4CFDF91CF911F910F91FF9008
:10163000EF90DF90CF90BF90AF9008950F931F93DE
:10164000CF93DF93EC0100E010E0888190E0081771
:1016500019070CF5ED81FE81C801880F991FE80F6D
:10166000F91F60817181FB018481882359F08034E6
:1016700021F48A81803461F405C0803649F48A817E
:10168000803631F480917109909172090E94580955
:101690000F5F1F4FDACF8A81803411F080E401C0E0
:1016A00080E68A83DF91CF911F910F9108951F9358
:1016B000CF93DF93182FC0E0D0E0E0917109F09153
:1016C000720980819181C817D90790F40680F7814B
:1016D000E02DCE01880F991FE80FF91F80819181BD
:1016E000FC012181211302C00E941E0B2196E5CF2F
:1016F000DF91CF911F91089580916C088330A1F004
:1017000028F4813041F0823051F008958430C9F0DE
:101710008530D9F0089580916D080C94570B809115
:101720006D0841E061E004C080916D0841E060E037
:101730000E94C7068FE99FE00197F1F700C0000003
:10174000089580916D080C94440780916E089091E3
:101750006E0840916D08977061E070E001C0660FFF
:101760009A95EAF783FB882780F90C94D1051F929C
:101770000F920FB60F9211240BB60F922F933F9337
:101780004F935F936F937F938F939F93AF93BF9389
:10179000EF93FF9399B180911D018923E1F599B1F0
:1017A00080911C01892339F090916A0880916B081F
:1017B000892B80936B0880916A08880F80936A0850
:1017C00080916A08811127C080916F0881110DC036
:1017D00080916B0880936C08E0916C08F0E0E95D03
:1017E000F94F808180936F080BC0E0916F08E15042
:1017F000E0936F08F0E080916B08E659F74F838320
:1018000080916F08811105C00E947C0B0E94960593
:1018100002C00E949005FF91EF91BF91AF919F91FF
:101820008F917F916F915F914F913F912F910F9089
:101830000BBE0F900FBE0F901F901895CF93DF93A4
:10184000EC018C81882349F081508C83811105C083
:10185000CE010E941E0B8B818C83DF91CF91089566
:10186000FC019181923009F43FC088F49923B9F0CA
:10187000913009F048C0E0917109F09172098485B6
:101880009585909382098093810984E0089593302F
:1018900031F09430C1F581E08093690834C09093B1
:1018A00061088681978190935E0880935D088281AC
:1018B0009381909358088093570810926008109273
:1018C0005F0880915B0890915C08892BF1F460912E
:1018D0005D0870915E0881E090E00E940110909395
:1018E0005C0880935B0811C0E7E1F8E0F09382099F
:1018F000E093810901900020E9F73197E751F84022
:1019000081E08E0F089580E008958FEF0895CF93C2
:10191000DF930E946C04EC0110925A08109259084F
:1019200060E071E00E944805882339F06091570813
:1019300070915808CE010E94BA0ACE01DF91CF9172
:101940000C941B030E94330940915D0850915E087E
:101950002EE031E061E070E080915B0890915C08DE
:101960000E94911220915D0830915E0882179307C2
:1019700029F40E94F00881E080936708089540915F
:101980005B0850915C08FC0170E0A0915F08B09189
:10199000600820915D0830915E08A217B307C8F473
:1019A0009F01281B390B261737079CF4A0915F086D
:1019B000B0916008A40FB51F21912C9320915F086E
:1019C000309160082F5F3F4F3093600820935F088D
:1019D000DCCF20915F083091600880915D08909184
:1019E0005E0828173907C8F080916108811103C08B
:1019F0000E94870C06C080916108833011F40E9418
:101A0000A20C80915B0890915C080E94B510109226
:101A10005C0810925B0881E0089580E00895CF9300
:101A2000DF9360918309635067FDA7C080918009AF
:101A3000CCE0D0E0C81BD109C957D64F80917F09AF
:101A40008D3209F088C0683009F095C083EC80932E
:101A500073098AE580933406109266082881822FE4
:101A6000807639F0CE010E94300C8F3F09F462C0BD
:101A700068C08A8110927C09998191110BC02F71E5
:101A800019F481E080937C0910927D092CE739E0FC
:101A900082E04BC0953019F48093840938C09630A9
:101AA00081F59B81913019F48EEC90E01FC092304B
:101AB00019F48CEB90E01AC09330F1F4811108C056
:101AC0008EE091E0909382098093810984E015C0B3
:101AD000813041F482EF90E09093820980938109F4
:101AE0008CE10BC0823041F480EE90E0909382094B
:101AF0008093810982E101C080E090E490936608C0
:101B000020C0983079F0993031F4809386092CE721
:101B100039E080E00AC081E09A3009F080E02CE7EB
:101B200039E003C026E839E081E030938209209350
:101B3000810907C0988197FD8E8190E8909366088F
:101B400007C09F81911104C09E81981708F4892FC6
:101B50008093330610C08091660887FF0CC0CE01C9
:101B60000E94BF0C8F3F21F48EE18093340603C0A6
:101B7000811110923306109283098091340684FFFC
:101B800048C0809133068F3F09F443C0C82F893085
:101B900008F0C8E08C1B809333069091730988E8A5
:101BA000892780937309CC2331F1409181095091A9
:101BB00082098091660886FF0AC0A4E7B9E0FA01AD
:101BC0009C2F84918D9331969150D9F708C0DA01FA
:101BD000E4E7F9E09C2F8D9181939150E1F72FEF8D
:101BE0002C0F30E02F5F3F4FCA01820F931F90935D
:101BF0008209809381096C2F84E799E00E94320E5C
:101C000064E06C0F6C3019F08FEF809333066093B3
:101C1000340684E199B1967031F48150D9F710926D
:101C2000840910927E09DF91CF910895E9E6F0E0F2
:101C3000808182608083E89A0895A82FB92F80E080
:101C400090E041E050EA609530E009C02D91822794
:101C50009795879510F084279527305EC8F36F5FBE
:101C6000A8F30895EADF8D939D930895CF93CFB79E
:101C7000CF93DF93C395499BE9F7499B0BC0499BE1
:101C800009C0499B07C0499B05C0499B03C0499BAC
:101C900001C089C06F93C0918009DD27C957D64F15
:101CA0002F9365E5499B03C02F916F91E6CF0F936A
:101CB0001F934F9320E040E15F9309B1067001FB51
:101CC00027F93F9350E03BE039C0167040642F770E
:101CD000012F5F5F1EC0406819B116702F775250F8
:101CE0001FC0406409B12F770670D1F15F5F00C05B
:101CF00023C0406219B12F77167091F15F5F00C069
:101D000025C006701027515012F45D5F000011507D
:101D100027952C3F19B1C8F6167001270150279559
:101D20002C3FC8F64227499309B1067010274F731C
:101D3000115027952C3FA8F64695469519B1167077
:101D400079F00127015027952C3F98F66B5A60F3E4
:101D5000315009B1B0F600C011E01CBB002717C01C
:101D60003B503195C31BD04011E01CBB0881033CA4
:101D7000F9F00B34E9F020917E091981110F12134B
:101D8000EDCF093651F10D3211F0013E39F70093D4
:101D900085093F915F914F911F910F912F916F9105
:101DA000CCB3C0FD67CFDF91CF91CFBFCF91189556
:101DB00020918509222369F310918309112339F5B4
:101DC00034303AF13093830920937F0910918009D0
:101DD0003BE0311B309380091CC000918309013026
:101DE000B4F40AE53091340634FD14C0009334068F
:101DF000C3E7D9E013C0052710E000C000000BB90D
:101E00001AC0052710E0221F1DC010E021C04AE5BE
:101E100002C032ED432FC4E1D0E032E01AB11660C7
:101E2000599A0BB11AB956E020E865E320FF05275F
:101E30000BB9279517951C3FF0F66695B8F7B1F7E3
:101E400020FF05270BB9279517951C3FD0F627953E
:101E5000179517FF052700001C3F0BB9B0F6299115
:101E60003A9519F7097F10918409110FC651D04096
:101E70000BB911F010937E0911E01CBB02601AB17E
:101E8000197F402F497F54E05A95F1F70BB91AB9E1
:101E90004BB97FCF0E94AC050E9410060E94C1057D
:101EA0000E947C088FE0809330091092690810929C
:101EB00067088BEA96E0909365088093640887EF43
:101EC00090E090936308809362080E946C04909362
:101ED0007209809371096EE071E00E9448058111DA
:101EE00006C080917109909172090E946B03E09184
:101EF0006408F0916508099560E070E080917109CF
:101F0000909172090E94BA0A0E94FC0511E001E05A
:101F10000E940F0D80916908811104C080916708AB
:101F2000882399F02FEF84E39CE02150804090407B
:101F3000E1F700C000008091690881110E948805C6
:101F40008091670881110E947C050E94030780919F
:101F50001208882319F08130A1F0DACF809130097E
:101F60000E948D07882351F0809171099091720928
:101F70000E9473020093120811E0CACF0E942F073B
:101F8000C7CF809130090E94BD07811103C0C0E016
:101F9000D0E024C0112321F0809130090E94440731
:101FA00010921208B5CF0680F781E02DCE01880F80
:101FB000991FE80FF91FE080F180F70181810E94ED
:101FC0008D07882351F0C7010E941E0CF701818103
:101FD0000E94BD078823D1F310E02196E09171099A
:101FE000F091720980819181C817D907E0F290CFF2
:101FF000EE0FFF1F0024001C0BBE0790F691E02D92
:1020000009940F931F93CF93DF93869F8001879F3F
:10201000100D969F100D1124C8010E941D10EC0197
:10202000009729F0A80160E070E00E943412CE0110
:10203000DF91CF911F910F9108950F931F93CF932D
:10204000DF938230910510F482E090E0E0919F09E7
:10205000F091A00920E030E0A0E0B0E0309719F165
:10206000408151810281138148175907C8F08417B4
:10207000950769F4109731F012960C931297139606
:102080001C9327C000939F091093A00922C021151B
:10209000310519F04217530718F49A01BD01EF01F9
:1020A000DF01F801DBCF21153105F9F0281B390BD1
:1020B0002430310580F48A819B816115710521F0FE
:1020C000FB019383828304C09093A00980939F09AE
:1020D000FE01329644C0FE01E20FF31F81939193FB
:1020E00022503109398328833AC020919D093091CB
:1020F0009E09232B41F42091370630913806309306
:102100009E0920939D0920913506309136062115B0
:10211000310541F42DB73EB74091390650913A064A
:10212000241B350BE0919D09F0919E09E217F307FE
:10213000A0F42E1B3F0B2817390778F0AC014E5F37
:102140005F4F2417350748F04E0F5F1F50939E09CD
:1021500040939D098193919302C0E0E0F0E0CF01AC
:10216000DF91CF911F910F910895CF93DF93009747
:1021700009F481C0FC01329713821282A0919F0959
:10218000B091A009109781F420813181820F931FB3
:1021900020919D0930919E092817390751F5F09338
:1021A0009E09E0939D0967C0ED0120E030E0CE1765
:1021B000DF0740F44A815B819E0141155105F1F032
:1021C000EA01F5CFD383C28340815181840F951FEB
:1021D000C817D90759F488819981840F951F0296F1
:1021E000918380838A819B8193838283211531052A
:1021F00029F4F093A009E0939F093DC0E901FB8316
:10220000EA8349915991C40FD51FEC17FD0761F47A
:1022100080819181840F951F0296E90199838883BB
:10222000828193819B838A83E0E0F0E012968D9116
:102230009C911397009719F0FD01DC01F7CF8D9168
:102240009C9111979D012E5F3F4F820F931F20910C
:102250009D0930919E092817390769F4309729F4B0
:102260001092A00910929F0902C013821282B093AB
:102270009E09A0939D09DF91CF9108956F927F925F
:102280008F929F92AF92BF92CF92DF92EF92FF9286
:102290000F931F93CF93DF93EC01009789F4CB0149
:1022A000DF91CF911F910F91FF90EF90DF90CF9032
:1022B000BF90AF909F908F907F906F900C941D1067
:1022C000FC01E60FF71F9C0122503109E217F307CA
:1022D00008F4A8C0D9010D911C9111970617170792
:1022E000B0F00530110508F49BC0C80104978617AB
:1022F000970708F495C002501109061B170B0193AC
:1023000011936D937C93CF010E94B51089C05B013E
:10231000A01AB10A4C01800E911EA0919F09B091A4
:10232000A009612C712CE12CF12C109709F446C006
:102330008D919C911197A815B905B1F56C0142E0FA
:10234000C40ED11CCA14DB0478F14C018A189B0816
:10235000640142E0C40ED11C1296BC9012971396F1
:10236000AC91B5E0CB16D10440F0B282A383918248
:102370008082D9016D937C9309C00E5F1F4F800F3F
:10238000911FF90191838083EB2DFA2FE114F10461
:1023900031F0D7011396FC93EE93129741C0F0935E
:1023A000A009E0939F093CC06816790608F43C0137
:1023B0007D0112960D90BC91A02DB7CF80919D0903
:1023C00090919E0988169906E1F466167706C8F47E
:1023D0008091350690913606009741F48DB79EB7EF
:1023E0004091390650913A06841B950BE817F9077E
:1023F000C8F4F0939E09E0939D09F901718360830D
:102400000FC0CB010E941D107C01009759F0A8015C
:10241000BE010E942B12CE010E94B510C70104C05C
:10242000CE0102C080E090E0DF91CF911F910F912B
:10243000FF90EF90DF90CF90BF90AF909F908F90E4
:102440007F906F9008959111089581548A5108F4F6
:10245000805E855A0895FB01DC0102C001900D9257
:1024600041505040D8F70895DC0101C06D934150B0
:102470005040E0F70895FB01DC018D910190801937
:102480000110D9F3990B0895FB01DC014150504034
:1024900048F001900D920020C9F701C01D924150F3
:1024A0005040E0F70895CF93DF93EC012B8120FF9C
:1024B00033C026FF0AC02F7B2B838E819F8101961C
:1024C0009F838E838A8190E029C022FF0FC0E8811C
:1024D000F9818081082E000C990B009719F4206275
:1024E0002B831AC03196F983E8830EC0EA85FB85F9
:1024F000099597FF09C02B81019611F080E201C078
:1025000080E1822B8B8308C02E813F812F5F3F4F5C
:102510003F832E83992702C08FEF9FEFDF91CF91EA
:1025200008958F929F92AF92BF92CF92DF92EF92D7
:10253000FF920F931F93CF93DF935B014A017901C1
:10254000D90113962C9121FF1DC0C0E0D0E0C81521
:10255000D905D9F08C016C01CA0CDB1CC8010C1523
:102560001D0571F00F5F1F4FD7011896ED91FC917B
:102570001997B701DC018C910995892B79F305C076
:102580002196E5CF80E090E001C0CE01DF91CF91B0
:102590001F910F91FF90EF90DF90CF90BF90AF9081
:1025A0009F908F9008950F931F93CF93DF93CDB794
:1025B000DEB72E970FB6F894DEBF0FBECDBF8C01ED
:1025C000FA0186E08C831A83098377FF02C060E0FA
:1025D00070E8CB0101979E838D83A901BF01CE01D5
:1025E00001960E9425134D815E8157FD0AC02F81FF
:1025F0003885421753070CF49A01F801E20FF31FD4
:1026000010822E960FB6F894DEBF0FBECDBFDF91BD
:10261000CF911F910F910895FB01238120FF12C0DC
:1026200026FD10C08F3F3FEF930761F082832F7D1F
:102630002064238326813781215031093783268303
:10264000992708958FEF9FEF08952F923F924F9211
:102650005F926F927F928F929F92AF92BF92CF9232
:10266000DF92EF92FF920F931F93CF93DF93CDB73B
:10267000DEB72C970FB6F894DEBF0FBECDBF6C014E
:102680007B018A01FC0117821682838181FFBEC112
:10269000CE0101964C01F6019381F70193FD8591DE
:1026A00093FF81917F01882309F4ACC1853239F40D
:1026B00093FD859193FF81917F01853229F4B601C5
:1026C00090E00E943715E7CF512C312C20E02032CA
:1026D000A0F48B3269F030F4803259F0833269F41F
:1026E00020612CC08D3239F0803339F4216026C04E
:1026F0002260246023C0286021C027FD27C030ED60
:10270000380F3A3078F426FF06C0FAE05F9E300DAD
:102710001124532E13C08AE0389E300D1124332E1D
:1027200020620CC08E3221F426FD6CC1206406C0EC
:102730008C3611F4206802C0883641F4F70193FD0D
:10274000859193FF81917F018111C1CF982F9F7D4A
:102750009554933028F40C5F1F4F9FE399830DC06D
:10276000833631F0833771F0833509F05BC022C0C6
:10277000F801808189830E5F1F4F44244394512CBC
:10278000540115C03801F2E06F0E711CF801A080F1
:10279000B18026FF03C0652D70E002C06FEF7FEFB0
:1027A000C5012C870E942C152C0183012C852F77C5
:1027B000222E17C03801F2E06F0E711CF801A080C4
:1027C000B18026FF03C0652D70E002C06FEF7FEF80
:1027D000C5012C870E9421152C012C852068222EF2
:1027E000830123FC1BC0832D90E048165906B0F4EA
:1027F000B60180E290E00E9437153A94F4CFF501DB
:1028000027FC859127FE81915F01B60190E00E942F
:10281000371531103A94F1E04F1A51084114510420
:1028200071F7E6C0843611F0893639F5F80127FFD3
:1028300007C060817181828193810C5F1F4F08C046
:1028400060817181072E000C880B990B0E5F1F4F62
:102850002F76722E97FF09C090958095709561959F
:102860007F4F8F4F9F4F2068722E2AE030E0A401E7
:102870000E946715A82EA81844C0853729F42F7E1A
:10288000B22E2AE030E025C0F22FF97FBF2E8F361E
:10289000C1F018F4883579F0B5C0803719F0883761
:1028A00021F0B0C02F2F2061B22EB4FE0DC08B2DB1
:1028B0008460B82E09C024FF0AC09F2F9660B92EED
:1028C00006C028E030E005C020E130E002C020E191
:1028D00032E0F801B7FE07C0608171818281938187
:1028E0000C5F1F4F06C06081718180E090E00E5F39
:1028F0001F4FA4010E946715A82EA818FB2DFF7773
:102900007F2E76FE0BC0372D3E7FA51450F474FE4B
:102910000AC072FC08C0372D3E7E05C0BA2C372D88
:1029200003C0BA2C01C0B52C34FF0DC0FE01EA0D66
:10293000F11D8081803311F4397E09C032FF06C059
:10294000B394B39404C0832F867809F0B39433FD15
:1029500013C030FF06C0B31498F43A0C532C5B1824
:1029600010C0B31470F4B60180E290E03C870E947E
:102970003715B3943C85F5CFB31418F43B1802C057
:102980005A2C312C34FF12C0B60180E390E03C8712
:102990000E9437153C8532FF17C031FD03C088E720
:1029A00090E002C088E590E0B6010CC0832F8678E5
:1029B00059F031FF02C08BE201C080E237FD8DE2A9
:1029C000B60190E00E943715A51438F4B60180E3F3
:1029D00090E00E9437155A94F7CFAA94F401EA0DBB
:1029E000F11D8081B60190E00E943715A110F5CF4E
:1029F000332009F450CEB60180E290E00E943715F2
:102A00003A94F6CFF6018681978102C08FEF9FEF4F
:102A10002C960FB6F894DEBF0FBECDBFDF91CF91DD
:102A20001F910F91FF90EF90DF90CF90BF90AF90EC
:102A30009F908F907F906F905F904F903F902F90DE
:102A40000895FC010590615070400110D8F7809501
:102A500090958E0F9F1F0895FC016150704001906A
:102A60000110D8F7809590958E0F9F1F08950F93B2
:102A70001F93CF93DF93182F092FEB018B8181FDDB
:102A800003C08FEF9FEF1EC082FF0FC02E813F81DA
:102A90008C819D812817390774F4E881F981CF0171
:102AA000019699838883108306C0E885F985812F74
:102AB0000995892B31F78E819F8101969F838E83A3
:102AC000812F902FDF91CF911F910F910895FA01DF
:102AD000AA27283051F1203181F1E8946F936E7F5D
:102AE0006E5F7F4F8F4F9F4FAF4FB1E03ED0B4E04E
:102AF0003CD0670F781F891F9A1FA11D680F791F8F
:102B00008A1F911DA11D6A0F711D811D911DA11D9F
:102B100020D009F468943F912AE0269F11243019AF
:102B2000305D3193DEF6CF010895462F4770405D4A
:102B30004193B3E00FD0C9F7F6CF462F4F70405DF9
:102B40004A3318F0495D31FD4052419302D0A9F754
:102B5000EACFB4E0A6959795879577956795BA954E
:102B6000C9F700976105710508959B01AC010A2E14
:102B700006945795479537952795BA95C9F7620FEB
:102B8000731F841F951FA01D0895262FF999FECF4E
:102B90001FBA92BD81BD20BD0FB6F894FA9AF99A7A
:102BA0000FBE019608950E94C515272F0C94C615D7
:042BB000F894FFCFC7
:102BB40000000001000000000000D600000000003A
:102BC400000300000000BF00AA0000002040808035
:102BD4004001100866080066080066080026060121
:102BE4006608002306036608006608006608006697
:102BF40008002006036608001D06031C060166087B
:102C0400006608006608001B060118060317060183
:102C14001606016608006608006608006608006675
:102C240008006608006608001306031206010F0672
:102C3400030C06030B06010806030506030206033C
:102C4400FF0503FC0503F90503F60503F30503F08B
:102C54000503EF0501EE0501ED0501EC0501EB05AA
:102C640001EA0501E90501E80501E70501E60501B9
:102C7400E50501E40501E30501E20501E10501E0E3
:102C84000501DF0501DE0501DB0503DA0501D705D2
:102C940003D40503D30501D00503CD0503CA0503F9
:102CA400C70503C40503C10503BE0503BB0503B87B
:102CB4000503B50503B20503AF0503AC0503A90578
:102CC40003A60503A30503A005039D05039A0503B5
:102CD4009705039405039105038E05038B0503886B
:102CE40005038505038205038105017E05037D0532
:102CF400017C050179050378050177050176050155
:102D040075050174050173050172050171050170F2
:102D140005016F05016E05016D05016C05016B056B
:102D2400016A050169050168050167050166050178
:102D34006505016405016305016205016105016022
:102D440005015F05015C0503590503560503530599
:102D5400035005036608004D050366080066080075
:102D64006608004C05014B05014A05014905014669
:102D740005034305034005033D05033A05036608BF
:102D8400006608003705033405033105032E0503E7
:102D94002D05012A05032705032405032105031E28
:102DA40005031B05031805031505031205030F0589
:102DB400030C05030B0501080503050503020503C0
:102DC400FF0403FC0403F90403F60403F30403F00F
:102DD4000403ED0403EA0403E70403E40403E10445
:102DE40003DE0403DB0403D80403D50403D2040381
:102DF400CF0403CC0403C90403C60403C30403C0FF
:102E04000403BD0403BA0403B70403B40403B10404
:102E140003AE0403AB0403AA0401A90401A804013A
:102E2400A70401A60401A50401A40401A30401A2AA
:102E34000401A10401A004019F04019E04019D0456
:102E4400019C04019B04019A040199040198040162
:102E540097040196040195040194040193040192DA
:102E640004019104018E04038B0403880403850484
:102E7400038204038104017E04037B0403780403B6
:102E84007504037204036F04036C0403690403668A
:102E940004036304036004035D04035A0403570436
:102EA400035404035104034E04034B040348040372
:102EB4004504034204033F04033C0403390403367A
:102EC40004033304033004032D04032A04032704F6
:102ED40003240403AFF66FAFE26FAFFA6FAFE26F94
:102EE400AFEA6FB9F579AFF46FAFF36FAFCB6FAFF4
:102EF400D56FAFD46FAFEB6FAFC96FAFCA6FAFF120
:102F04006FAFD16FAFCD6FAFE96FAFE16FAFD26F7E
:102F1400AFF76FAFD56FB9C679AFC66FAFE46FAF18
:102F2400C56FAFD36FAFF56FAFF26FAFCC6FAFECD0
:102F34006FE7AFCE6FAFF66FB9E379AFDD6FB9C5A9
:102F440079E1CBFAC9FBF3F2E9CAF7CDF4FCE4D595
:102F5400ECD4CCEBD3EAF1D2E2E3D1B9CE79AFE34E
:102F64006FAFE26FAFFA6FAFE26FAFEA6FB9F579A7
:102F7400AFF46FAFF36FAFCB6FAFD56FAFD46FAFAD
:102F8400EB6FAFC96FAFCA6FAFF16FAFD16FAFCD9A
:102F94006FAFE96FAFE16FAFD26FAFF76FAFD56FC0
:102FA400B9C679AFC66FAFE46FAFC56FAFD36FAFBC
:102FB400F56FAFF26FAFCC6FAFEC6FE797D9579760
:102FC400DB57B9D07997C257AFDB6FAFC36FAFDAB6
:102FD4006FAFC26FAFD96FAFC16FAFDF6FC0B9DE74
:102FE4007997DC57B9F87997C757B9C879B9D879B7
:102FF400B9F079B9E879B9E079D8F0E8E0AFC76F0A
:10300400AFCE6FAFF66FB9E379AFDD6FB9C579E1D4
:10301400CBFAC9FBF3F2E9CAF7CDF4FCE4D5ECD45E
:10302400CCEBD3EAF1D2E2E3D1B9CE79CFF6B9D67B
:1030340079C6B9ED79B9E179B9CB79B9FA79B9C970
:1030440079B9FB79B9F379B9F279B9E979B9CA7976
:10305400B9F779B9CD79B9F479B9FC79B9E479B921
:10306400D579B9EC79B9D479B9CC79B9EB79B9D343
:1030740079B9EA79B9F179B9D279B9E279B9E37967
:10308400B9D179F5B9FE79B9E579EEB9FD79D6ED1D
:10309400C4DBC3DAC2D9C1DFC7DCFEE5DDFDC5CEC2
:1030A400B9C479B9DB79B9C379B9DA79B9C279B96B
:1030B400D979B9C179B9DF79B9C779E797C357978E
:1030C400DA57D097C157C0DE97C457F8C8B9DE792C
:1030D400B9C87997DF57FF000101010102FCFDFE29
:1030E400FF1CCFFF5A0000A109200060406040008F
:1030F4000C0A202A2A2A2A2A206B65796D616E36E9
:10310400342076657273696F6E20312E34207265B7
:10311400616479202A2A2A2A2A0A0A202020206E79
:103124006F20636F6E66696775726174696F6E2074
:10313400666F756E6420696E20656570726F6D0AC6
:103144002020202020207573696E672066616C6CD6
:103154006261636B20636F6E66696775726174691F
:103164006F6E0A0A202020202020205F763A2074E7
:10317400797065206669726D776172652076657213
:1031840073696F6E0A202020202020205F623A207D
:10319400656E74657220626F6F746C6F61646572C2
:1031A4000A202020202020205F663A207465737452
:1031B400206372797374616C206672657175656ED3
:1031C40063790A202020202020205F743A2074791B
:1031D40070652074686973206D6573736167650A2F
:1031E4000A72656164792E0A000C0A202A2A2A2AA6
:1031F4002A20206B65796D616E36342066726571A4
:1032040075656E6379207465737420202A2A2A2ACE
:103214002A0A0A69662074686520666F6C6C6F7789
:10322400696E672074656E20646F747320617265C3
:10323400206E6F742074797065640A7769746820ED
:1032440061626F7574206F6E65207365636F6E6461
:103254002064656C617920696E20626574776565A8
:103264006E2C0A636865636B2061746D656C2066FF
:103274007573657320616E642F6F72206372797346
:1032840074616C20636972637569740A006669729B
:103294006D7761726520312E34204E6F762031387F
:1032A40020323031362031363A31373A3235003037
:1032B40030303030303030006120006220000A0AA3
:0232C400000008
:020000021000EC
:10E000007EC00000BFC00000A3C00000A1C000008F
:10E010009FC000009DC000009BC0000099C0000090
:10E0200097C0000095C0000093C0000091C00000A0
:10E030008FC000008DC000008BC0000089C00000B0
:10E0400087C0000085C0000083C0000081C00000C0
:10E050007FC000007DC000007BC0000079C00000D0
:10E0600077C0000075C0000073C0000071C00000E0
:10E070006FC000006DC000006BC0000069C00000F0
:10E0800067C0000065C0000063C00000BBBEEC2D8F
:10E09000FD2DB7B6B0FCFDCF27BFE895B7B6B0FCF5
:10E0A000FDCF21E1B7B6B6FCF4CF08950902120006
:10E0B000010100803209040000000000000012018C
:10E0C0001001FF000008C016DC050201010200017A
:10E0D0000E035500530042006100730070001C03E2
:10E0E0007700770077002E006600690073006300F8
:10E0F00068006C002E00640065000403090411240C
:10E100001FBECFEFD0E4DEBFCDBF24B7D0E4CEEF4B
:10E110003991303F399109F03FEF30933E01209320
:10E120003D0111E0A0E0B1E0ECEBF9EE01E00BBF46
:10E1300002C007900D92A630B107D9F721E0A6E002
:10E14000B1E001C01D92AD33B207E1F78CD134C408
:10E1500057CFA82FB92F80E090E041E050EA6095BA
:10E1600030E009C02D9182279795879510F084277C
:10E170009527305EC8F36F5FA8F30895EADF8D93AB
:10E180009D930895CF93CFB7CF93DF93C395499BCA
:10E19000E9F7499B0BC0499B09C0499B07C0499BB4
:10E1A00005C0499B03C0499B01C089C06F93C091C2
:10E1B0002001DD27C95DDE4F2F9365E5499B03C034
:10E1C0002F916F91E6CF0F931F934F9320E040E183
:10E1D0005F9309B1067001FB27F93F9350E03BE0E4
:10E1E00039C0167040642F77012F5F5F1EC04068F2
:10E1F00019B116702F7752501FC0406409B12F77A4
:10E200000670D1F15F5F00C023C0406219B12F7763
:10E21000167091F15F5F00C025C006701027515045
:10E2200012F45D5F0000115027952C3F19B1C8F61C
:10E2300016700127015027952C3FC8F642274993B5
:10E2400009B1067010274F73115027952C3FA8F67F
:10E250004695469519B1167079F00127015027951A
:10E260002C3F98F66B5A60F3315009B1B0F600C0FC
:10E2700011E01CBB002717C03B503195C31BD04099
:10E2800011E01CBB0881033CF9F00B34E9F020914C
:10E290001E011981110F1213EDCF093651F10D3204
:10E2A00011F0013E39F7009325013F915F914F91A5
:10E2B0001F910F912F916F91CCB3C0FD67CFDF916C
:10E2C000CF91CFBFCF91189520912501222369F3DB
:10E2D00010912301112339F534303AF130932301A1
:10E2E00020931F01109120013BE0311B309320014E
:10E2F0001CC0009123010130B4F40AE53091010102
:10E3000034FD14C000930101C3E1D1E013C005271F
:10E3100010E000C000000BB91AC0052710E0221F52
:10E320001DC010E021C04AE502C032ED432FC4E118
:10E33000D0E032E01AB11660599A0BB11AB956E022
:10E3400020E865E320FF05270BB9279517951C3FAB
:10E35000F0F66695B8F7B1F720FF05270BB92795BA
:10E3600017951C3FD0F62795179517FF0527000036
:10E370001C3F0BB9B0F629913A9519F7097F109116
:10E380002401110FC651D0400BB911F010931E019A
:10E3900011E01CBB02601AB1197F402F497F54E085
:10E3A0005A95F1F70BB91AB94BB97FCFDC01139627
:10E3B0003C911397F32F14962C911497E22F1296F9
:10E3C0009C911297903339F42370E22FF0E0EE5FC6
:10E3D000FE4F80810895983529F431110EC0E1E097
:10E3E000F0E006C0903599F431110CC0E0E0F0E0A7
:10E3F00089E08093570084910895383091F5E3E0E7
:10E40000F0E0F6CF383069F5E2E0F0E0F1CF90329D
:10E4100041F4CF01A0E0B0E0880F991FAA1FBB1FF5
:10E420000CC0983271F4CF01A0E0B0E0880F991FC2
:10E43000AA1FBB1F0196A11DB11DABBFFC01879197
:10E440000895903A11F4CF0189C2903C29F41596B1
:10E450006C91CF0190D205C09F3F19F481EF80935A
:10E46000110180E008951AB881E08BB985BF92E070
:10E4700095BFE0E0F1E7A89531979040E1F704B649
:10E4800003FE0EC08EEF9FE071D2C1E0803B904B47
:10E4900009F0C0E06FEF7FEF8EEF9FE07AD208C007
:10E4A00004B601FE04C0C9B1C170C82701C0C0E0F4
:10E4B00014BEC1110CC0F894519A1BB81DBA109229
:10E4C000690081E085BF15BEE0E0F0E009958EEFC0
:10E4D0008093110114BE0FB6F894A8958091600046
:10E4E000886180936000109260000FBE8091690087
:10E4F000826080936900E89A519A8CE0E0E0F5E34D
:10E50000A89531978040E1F75198789481EF8093F6
:10E51000110110912301135017FD74C18091200146
:10E52000CCE0D0E0C81BD109C95DDE4F80911F014E
:10E530008D3209F0C0C0183009F062C183EC8093BD
:10E5400013018AE580930101109212013881832F13
:10E5500080769981882309F43FC046E051E05093CA
:10E56000220140932101933031F4CE011FDF8093CB
:10E57000090184E096C0953009F492C09A3009F4FC
:10E580008FC08CEF890F8630E0F44A815B81509315
:10E590000E0140930D01993039F48C819D81909347
:10E5A000100180930F0114C08E8180930C012D8186
:10E5B000227020930B0190930A0137FD6DC08FEFFD
:10E5C0006BC080911101923029F48E7F80931101EC
:10E5D00080E067C08160FACF8A8110921C0191119E
:10E5E00006C010921D012CE131E082E050C0953050
:10E5F00019F4809324013DC09630A9F59B81913098
:10E6000019F48EEB90EE04C0923041F48CEA90EE57
:10E61000909322018093210182E121C09330F1F493
:10E62000811108C08AEF90EE90932201809321011E
:10E6300084E015C0813041F48EED90EE909322017C
:10E64000809321018CE10BC0823041F480ED90EE8B
:10E6500090932201809321018EE001C080E090E43C
:10E66000909312011EC0983079F0993031F4809364
:10E6700026012CE131E080E00AC081E09A3009F007
:10E6800080E02CE131E003C026E231E081E030930C
:10E6900022012093210105C090E89093120108C047
:10E6A00081E09F81911104C09E81981708F4892F01
:10E6B00080930001A5C08091120187FFA1C0009145
:10E6C0000C01011708F4102F011B00930C01F12C11
:10E6D000F11608F091C080910A018730A0F06E0118
:10E6E000FFEFCF1ADF0A688180910D0190910E0132
:10E6F0009C012F5F3F4F30930E0120930D013BD1C2
:10E70000F394E601E5CF80910D0190910E01A09167
:10E710000F01B09110018115904EA140B10508F094
:10E720006DC0F394F394F89440910D0150910E0153
:10E7300060910F01709110012991399181E00901D7
:10E74000FA0160935B0080935700E8951124789458
:10E7500080910D0190910E01A0910F01B0911001D7
:10E760000296A11DB11D80930D0190930E01A093FF
:10E770000F01B0931001882351F00111A9CFF116B8
:10E7800008F4A6CF80910B01882309F4A1CFF89457
:10E7900080910D0190910E01A0910F01B091100197
:10E7A0000297A109B10923E0FC01A0935B0020932B
:10E7B0005700E895789407B600FCFDCFF894809157
:10E7C0000D0190910E01A0910F01B09110010297DF
:10E7D000A109B10925E0FC01A0935B00209357003B
:10E7E000E895789407B600FCFDCFF89481E180931A
:10E7F0005700E89578946CCF011102C01092000187
:10E80000109223018091010184FF7EC0809100015C
:10E810008F3F09F479C0C82F893008F0C8E08C1BFD
:10E82000809300019091130188E889278093130158
:10E83000CC2309F48DC08091120187FF37C08091ED
:10E840000C018C1708F4C82F8C1B80930C01B0901E
:10E850000A01D0E004E111E0CD1709F449C0C090ED
:10E860000D01D0900E01E0900F01F090100186E0B4
:10E870008B1530F480910D0190910E016FD003C083
:10E88000EBBEF6018791F80180830F5F1F4FFFEF0A
:10E89000CF1ADF0AEF0AFF0AC0920D01D0920E01D3
:10E8A000E0920F01F0921001DF5FD6CFA09121011D
:10E8B000B091220186FF11C024E131E08C2FAD011F
:10E8C00060E070E061606BBFFA014791F90141932C
:10E8D0009F011196815099F707C0E4E1F1E08C2F78
:10E8E0009D9191938150E1F7B0932201A093210172
:10E8F0006C2F84E191E042DCCC5FCC3019F08FEFDB
:10E9000080930001C093010184E199B1967031F4C4
:10E910008150D9F71092240110921E0180911101AB
:10E92000803130F0489B0FC080911101805109C0A7
:10E93000489909C080911101823028F0809111011D
:10E94000825080931101809111018111E2CDB3CDEC
:10E9500060E084E191E012DCC4E0D1CFF999FECF10
:10E9600092BD81BDF89A992780B50895A8E1B0E0DD
:10E9700042E050E013C0262FF999FECF1FBA92BD96
:10E9800081BD20BD0FB6F894FA9AF99A0FBE019690
:10E990000895F1DF272FF0CFDC01CB01FC01F999BD
:10E9A000FECF06C0F2BDE1BDF89A319600B40D92DB
:0CE9B00041505040B8F70895F894FFCF94
:06E9BC00FF5A1E97050042
:040000031000E00009
:00000001FF
